:020000040800F2
:1000000000070020F10100086D24000825240008E5
:100010004D2400082524000845240008F3010008A9
:10002000F3010008F3010008F30100086D34000833
:10003000F3010008F3010008F3010008F3010008D0
:10004000F3010008F3010008F3010008F3010008C0
:10005000F3010008F30100080142000829420008EA
:100060005142000879420008A1420008F30100084B
:10007000F3010008F3010008F3010008F301000890
:10008000F3010008F3010008F3010008D923000878
:100090000524000815240008F3010008C9420008DF
:1000A000F3010008F3010008F3010008F301000860
:1000B0009D430008F3010008F3010008F301000864
:1000C000F3010008F3010008F3010008F301000840
:1000D000F3010008F3010008F3010008F301000830
:1000E0002D430008F3010008F3010008F3010008A4
:1000F000F3010008F3010008F3010008F301000810
:10010000F3010008F3010008F3010008F3010008FF
:10011000F3010008F3010008F3010008F3010008EF
:10012000F3010008F3010008F3010008F3010008DF
:10013000F3010008F3010008F3010008F3010008CF
:10014000F3010008F3010008F3010008F3010008BF
:10015000F3010008F3010008F3010008F3010008AF
:10016000F3010008F3010008F3010008F30100089F
:10017000F3010008F3010008F3010008F30100088F
:10018000F3010008F3010008F3010008F30100087F
:10019000F3010008F3010008F3010008F30100086F
:1001A000F3010008F3010008F3010008F30100085F
:1001B000F3010008F3010008F3010008F30100084F
:1001C000F3010008F3010008F3010008F30100083F
:1001D000F3010008F3010008F3010008F30100082F
:1001E000B90F00080000000000000000000000003F
:1001F00002E000F000F8FEE772B6374880F30888A6
:10020000364880F3098836483649086040F20000D5
:10021000CCF200004EF63471CEF200010860BFF35C
:100220004F8FBFF36F8F40F20000C0F2F0004EF628
:100230008851CEF200010860BFF34F8FBFF36F8F7C
:100240004FF00000E1EE100A4EF63C71CEF20001D4
:100250000860062080F31488BFF36F8F03F0E6FD7B
:1002600003F078FE4FF055301F491B4A91423CBFC6
:1002700041F8040BFAE71D49184A91423CBF41F886
:10028000040BFAE71A491B4A1B4B9A423EBF51F82E
:10029000040B42F8040BF8E700201849184A914271
:1002A0003CBF41F8040BFAE703F0C4FD03F0A6FEDF
:1002B000144C154DAC4203DA54F8041B8847F9E797
:1002C00000F042F8114C124DAC4203DA54F8041B12
:1002D0008847F9E703F0ACBD0007002000230020A9
:1002E0000000000808ED00E00001002000070020E9
:1002F000884700080023002080230020802300205E
:10030000504D0020E0010008E4010008E40100086D
:10031000E40100082DE9F04F2DED108AC1F80CD052
:10032000C3689D46BDEC108ABDE8F08F002383F3BF
:1003300011882846A047002003F0F4F9FEE703F0F7
:100340007DF900DFFEE70000F8B500F047FE03F09E
:1003500007FD074603F056FD0546C0BB294B9F42EB
:1003600035D001339F4235D0274B27F0FF029A4208
:1003700033D1F8B200F03EFC2E4642F2107400F089
:100380003FFC08B10024264601F04CF948B3032095
:1003900000F03EF80024264635B11C4B9F4203D0A6
:1003A00003F028FD00242646002003F0E3FC0EB1F4
:1003B00000F044F800F090FC02F060F80546C4B983
:1003C00000F0D2FC4FF47A7003F0B2F9F7E72E4652
:1003D0000024D4E704460126D1E7064641F28834DA
:1003E000CDE741F288339C4204BF4FF47A74012672
:1003F000D2E702F043F8431BA342E1D900F01EF814
:10040000DAE700BF010007B0000008B0263A09B0E3
:10041000084B187003280CD8DFE800F00805020824
:10042000022000F039BE022000F02CBE024B002258
:100430005A607047802300208423002010B501F00B
:10044000F1F830B1204B03221A70204B00225A6081
:1004500010BD1F4B1F4A1C4619680131F8D00433E8
:100460009342F9D162681C4B9A42F1D91B4B9B68AD
:1004700003F1006303F580339A42E9D203F08EFC66
:1004800003F0A0FC002000F0C3FD0220FFF7C0FF36
:10049000134B1A6C00221A64196E1A66196E596C85
:1004A0005A64596E5A665B6E72B64FF0E023302183
:1004B000C3F8084DD4E9003281F311889D4683F3D7
:1004C00008881047C4E700BF802300208423002051
:1004D0000000010820000108FFFF000800230020A1
:1004E00000380240094A136849F2690099B21B0CAE
:1004F00000FB01331360064B186844F2506182B26E
:10050000000C01FB0200186080B270471823002025
:100510001423002010B500211022044600F0D8FD5D
:10052000034B03CB206061601868A06010BD00BF62
:10053000107AFF1F2DE9F041ADF54C7D0DF12C082F
:100540006AAC40F2751207460D460CA80021C8F8A7
:10055000001000F0BDFD4FF4C4720021204600F0F1
:10056000B7FD01F08BFF274B4FF47A72B0FBF2F02E
:10057000186093E80700022384E807000DF5E57092
:100580002382FFF7C7FF47F217131F49238407A8E9
:1005900004F010F80F2384F832310DF2DB2207ABA0
:1005A0000DF1240C1E4603CE6645106051603346A3
:1005B00002F10802F6D130681060B188B379937106
:1005C000918020464146012200F0CEFD0023039396
:1005D000AB7E029305F11903019380B20123CDE9AB
:1005E00004800093E97E05A3D3E90023384602F096
:1005F0000DFB0DF54C7DBDE8F08100BF9E6AC42166
:10060000818A46EE8C230020C44500082DE9F04184
:100610002C4C237ADAB080460D465BBB27A92846CE
:1006200000F0C4FE0746002842D19DF89D60C82E08
:100630003ED801464FF4A662204600F049FD4FF433
:100640008073C4F8F8314FF40073C4F80C334FF4DE
:100650004073C4F8203432460DF19E0104F10900C4
:1006600000F024FD26449DF89C30777223720BB96C
:10067000EB7E23728122002106AC27A800F028FD22
:100680000122214627A800F0D7FE00230393AB7E6A
:10069000029305F1190380B201932823CDE90440A8
:1006A0000093E97E05A3D3E90023404602F0AEFAA9
:1006B0005AB0BDE8F08100BFAFF3008026417272EE
:1006C000DF25D7B7B0440020F0B5254E4FF48A752A
:1006D00005FB0065F1B096F8D83085F8DC300024D1
:1006E000D822214685F8E8403AA800F0F1FC06F14E
:1006F000090000F0E5FCD5F8E4308DF8F000C2B256
:1007000006AF06F109010DF1F100CDE93A3400F030
:10071000CDFC394601223AA800F0C4FE80B2CDE9F2
:10072000047008230127CDE9023706F1D8030193AD
:1007300030230093317A0B4807A3D3E9002302F05A
:1007400065FAA04206DD01F099FEC5F8E0003846E2
:1007500071B0F0BD2046FBE778F6339F93CACD8D8C
:10076000B0440020A43300202DE9F0411D4D1E4E61
:100770001E4F86B0284602F075FA034658B300248F
:10078000CDE90344ADF81440027B8DF8142099683C
:100790004068029403AA03C21B68DFF8548043F048
:1007A0000043029301F06CFE821941F100030094B2
:1007B00002A9384601F014F9A04205DD284602F0EE
:1007C00055FA88F80040D5E798F80030072B05D88F
:1007D000013388F8003006B0BDE8F081014802F02E
:1007E00045FAF8E7A433002040420F00D833002038
:1007F000E549002070B50D4614461E4602F062F928
:1008000050B9022E10D1012C0ED112A3D3E900232E
:10081000C5E90023012007E0282C10D005D8012CC1
:1008200009D0052C0FD0002070BD302CFBD10BA3BC
:10083000D3E90023ECE70BA3D3E90023E8E70BA3FC
:10084000D3E90023E4E70BA3D3E90023E0E700BFEB
:10085000AFF30080401DA12026812A0B78F6339F3C
:1008600093CACD8D9E6AC421818A46EE264172725A
:10087000DF25D7B7F017304A39059E5638B50546FB
:100880000E4C0021013500F0E5FBA4F82C55B4F81E
:100890002C0500F0C7FB78B1B4F82C0500F0D2FBB2
:1008A000014648B9B4F82C0500F0D4FBB4F82C3557
:1008B0000133A4F82C35EAE738BD00BFB04400206E
:1008C00010B50A4B0A4A1A6003F5805393F860206A
:1008D0003AB9DC6D2CB1204600F022FF204603F02F
:1008E000A9FDBDE81040034800F01ABFD83300202E
:1008F00010460008204400202DE9F04F8FB000AFD3
:1009000005460C4602F0DEF8002849D1237E022B72
:100910001BD1E38A012B18D101F0B0FD0646FFF789
:10092000E1FD03464FF4C870DFF8C482B3FBF0F278
:1009300006F5167602FB103316FA83F3C8F800307A
:10094000E37E33B9A34B00221A703C37BD46BDE8A5
:10095000F08F07F12401204600F0DCFC0028F4D1E0
:1009600007F11400FFF7D6FD97F8264007F11401B0
:10097000224607F1270003F0A7FD0028E2D10F2C43
:1009800008D8944B1C70D8F80030A3F51673C8F83B
:100990000030DAE797F82410284602F08BF8D4E705
:1009A000E38A282B2BD010D8012B23D0052BCCD1B8
:1009B000BFF34F8F8849894BCA6802F4E062134342
:1009C000CB60BFF34F8F00BFFDE7302BBDD1844E0E
:1009D000E17E327A9142B8D1607E3146002291F8B0
:1009E000DC50854200F0A5800132042A01F58A71AD
:1009F000F5D1AAE721462846FFF79CFDA5E7214649
:100A00002846FFF703FEA0E7B2F8EC507B6005F143
:100A100003094FEA99094FEA8902D11DC908A8EBD9
:100A2000C1039D46EB460021584600F051FB04F1FE
:100A3000EE012A463144584600F038FB7B6813B972
:100A4000012000F0E5FA96F8D20000F0EBFA044637
:100A500030B9307200F006FB204600F0D9FAB1E060
:100A6000D6F8D4203AB996F8D200B6F82C258242AE
:100A700001D8FFF703FFD6F8D4202A44944208D2C5
:100A800096F8D200B6F82C250130824201D8FFF743
:100A9000F5FE70685FFA89F2594600F021FB08B94B
:100AA000C54679E0726896F8D2002A447260D6F89A
:100AB000D42005EB0209C6F8D49000F0B3FA8145C2
:100AC00009D396F8D220D6F8D4000132001B86F85C
:100AD000D220C6F8D400FF2D0FD80024347200F0C5
:100AE000C1FA204600F094FA00F09CFD3D4B1881BD
:100AF00008B9FFF7A3FCC54627E7BB6896F8D900FD
:100B00000AFB0362FB68D2F8E41082F8E83001F5D2
:100B10008061C2F8E030C2F8E410FFF7D5FDFFF7BE
:100B200023FE96F8D920013202F0030286F8D9207C
:100B3000B6E74FF48A7A0AFB02F505F1EA0131447F
:100B4000204600F0E1FCF86000287FF4FEAE35445A
:100B5000012285F8E82001F091FCD5F8E020D6EDDF
:100B6000007ADFED216A801A192838BF192040F673
:100B7000B832904228BF1046B8EE677A07EE900A66
:100B8000F8EEE77A67EEA67ADFED186AE7EE267AE6
:100B9000FCEEE77AC6ED007A96F8D930BB60BA6809
:100BA00073680AFB02F4321992F8E81059B1D2F8CE
:100BB000E4108B42E8463FF427AF002182F8E810AA
:100BC000C2F8E010C5467368064A9B0A01331381D8
:100BD000BBE600BF9D33002000ED00E00400FA05F5
:100BE000B04400208C230020CDCCCC3D6666663F0F
:100BF000A0330020014B1870704700BF98230020DD
:100C000030B54FF000542B4B22689A4285B007D084
:100C100003F002F9044620BB0024204605B030BD95
:100C2000254B627D25481A70237D03724FF4807333
:100C3000C0F8F8314FF40073C0F80C3300254FF4BE
:100C40004073C0F820341E49C0F8E450C92209306E
:100C500000F02CFA2046E022294600F039FA01245F
:100C6000DBE7184A184D136C43F000731364AA6D48
:100C7000164B9A42D0D12B6E013B7E2BCCD8144A16
:100C800007CA01AB83E807001846032100F098FC6F
:100C90006B6D83424FF00003BED12A6D8A4201BFC3
:100CA000AB65054B2A6E1A7003BF0A4BEA6D1A60DA
:100CB0001C46B2E79AAD44C598230020B0440020FA
:100CC0001600002000380240006600405041A0B0ED
:100CD000586600401023002037B51A4D00F0A2FCE2
:100CE00002236B71184B288119681848012201F002
:100CF00061FA00230193164B164900931648174BCF
:100D00004FF4805201F0AEFE154B197811B1124824
:100D100001F0D0FE01F0B2FB0446FFF7E3FB4FF415
:100D2000C873B0FBF3F202FB130304F5167010FA5C
:100D300083F00C4B186003F065F808B10F232B818A
:100D400003B030BD8C23002010230020D8330020B6
:100D5000F50700089C230020A4330020F9080008B0
:100D600098230020A03300202DE9F04F2DED028BB9
:100D70000FF23829D9E90089834C93B00BAE9FED6F
:100D80007E8BFFF7F1FC814FDFF828A200230A9346
:100D9000ADF834300B9373604FF0000B5B468DED74
:100DA000008B01250DF11D0207A938468DF81C5056
:100DB0008DF81DB001F0ACF99DF81C30002B40F00F
:100DC000A580204601F07EFE0646002845D1704FE2
:100DD00001F054FB3B6898423FD301F04FFB824641
:100DE000FFF780FB4FF4C873B0FBF3F202FB130371
:100DF0000AF5167010FA83F03860664F97F800B065
:100E0000CBF1100ABBF1000F14BF33462B465FFA3B
:100E10008AFA0EA88DF82830FFF77CFBBAF1060F8E
:100E200028BF4FF0060A0EAB03EB0B0152460DF143
:100E3000290000F03BF90AAB0393182302930AF14F
:100E40000102554BD2B2CDE90053049220464CA387
:100E5000D3E9002301F07CFE3E7001F00FFB4F4A06
:100E60004F4D1368C31AB3F57A7F2ED3106001F08B
:100E700007FB02460B46204601F002FF204601F028
:100E800021FE10B32B7A474E002B14BF03230223FD
:100E9000737101F0F3FA0EAF4FF47A730122B0FBD5
:100EA000F3F039463060304600F00CFA1823029314
:100EB0003D4B019380B240F25513CDE9037000938E
:100EC00042464B46204601F043FE2B7A93B101F097
:100ED000D5FA002607464FF48A7A95F8D9003044AF
:100EE00000F003000AFB005393F8E82092B30136A8
:100EF000042EF2D1C82002F01BFC2B7A002B7FF4C9
:100F00003DAF13B0BDEC028BBDE8F08FDAF81430C2
:100F100083F48073CAF81430594610220EA800F0EA
:100F2000D7F80DF11E0308AA0AA9384600F058FEAA
:100F300096E803000FAB83E803009DF834308DF88A
:100F400044300A9B0E930EA9DDE90823204602F0E7
:100F50006BF821E7D3F8E02042B12B68FA2B38BFB9
:100F6000FA23BA1A0533B2EB430FC0D3FFF7ACFB39
:100F70000028BCD1BEE700BF000000000000000058
:100F8000401DA12026812A0BA4330020D833002045
:100F9000A03300209D3300209C330020E049002036
:100FA000B04400208C230020E4490020F1C6A7C1F2
:100FB000D068080F0008024008B5054800F0ACFEF4
:100FC000BDE80840034A0449002003F02DBA00BFE1
:100FD000D8330020204A0020C108000870B502F074
:100FE0005FFD094E094D3080002428683388834214
:100FF00008D902F04FFD2B6804440133B4F5803F5B
:101000002B60F2D370BD00BF144A0020E8490020D5
:1010100002F0F6BD00F10060920000F5803002F0B1
:1010200085BD0000054B1A68054B1B889B1A83423F
:1010300002D9104402F02EBD00207047E84900207C
:10104000144A0020024B1B68184402F02BBD00BF5D
:10105000E8490020024B1B68184402F03BBD00BF6A
:10106000E8490020064991F8243033B10023086A8A
:1010700081F824300822FFF7CDBF0120704700BF60
:10108000EC490020022802BF024B4FF480729A61A3
:10109000704700BF00080240022802BF024B4FF019
:1010A00080729A61704700BF0008024010B50023AB
:1010B000934203D0CC5CC4540133F9E710BD000067
:1010C00003460246D01A12F9011B0029FAD17047D3
:1010D00002440346934202D003F8011BFAE770472B
:1010E0002DE9F8431F4D144695F8242007468846FD
:1010F00052BBDFF870909CB395F824302BB92022B6
:10110000FF2148462F62FFF7E3FF95F82400C0F166
:101110000802A24228BF2246D6B24146920005EB01
:101120008000FFF7C3FF95F82430A41B1E44F6B2DD
:10113000082E17449044E4B285F82460DBD1FFF711
:1011400091FF0028D7D108E02B6A03EB820383428A
:10115000CFD0FFF787FF0028CBD10020BDE8F88370
:101160000120FBE7EC4900202DE9F8430D46044639
:1011700000219046284640F27912FFF7A9FF234646
:1011800020220021284601F0F1FE231D0222202109
:10119000284601F0EBFE631D03222221284601F0C0
:1011A000E5FEA31D03222521284601F0DFFE04F100
:1011B000080310222821284601F0D8FE04F110036C
:1011C00008223821284601F0D1FE04F1110308223B
:1011D0004021284601F0CAFE04F1120308224821EA
:1011E000284601F0C3FE04F11403202250212846B2
:1011F00001F0BCFE04F1180340227021284601F0E2
:10120000B5FE04F120030822B021284601F0AEFE0D
:1012100004F121030822B821284601F0A7FE04F1B9
:101220002207C0263B46314608222846083601F0F0
:101230009DFEB6F5A07F07F10107F3D1314604F119
:1012400032030822284601F091FE94F8326000270C
:1012500004F13309F900BE4201F5A4711FD8F7006B
:1012600007F5A476B8F1000F08D1314604F599735B
:101270000722284601F07AFE07F24F1694F8320151
:10128000502828BF5020074604EB0009B046A1456E
:101290000DD106EBC7000730C008BDE8F88309EBA5
:1012A00007030822284601F061FE0137D2E704F265
:1012B000331341460822284601F058FE08F1080879
:1012C0000134E4E713B504460846002101602346D3
:1012D000C0F803102022019001F048FE0198231D60
:1012E0000222202101F042FE0198631D03222221E7
:1012F00001F03CFE0198A31D0322252101F036FEDA
:10130000019804F108031022282101F02FFE072084
:1013100002B010BDF7B5047F05460E462CB1838A96
:10132000122B02D9012003B0F0BD00231946072279
:101330000096284601F0DEFC731C00930122002376
:101340000721284601F0D6FCD4B9B31C009305222E
:1013500023460821284601F0CDFC0D24B378102B3C
:10136000E0D83746B278BB1B934210D32B7FA88AB4
:101370000734E408B3B9844294BF00200120D2E7C7
:10138000AB8ADB00083BDB08B3700824E6E7FB1CF4
:101390000093214600230822284601F0ABFC0834C4
:1013A0000137DFE7201A18BF0120BCE7F7B5047F3B
:1013B00005460E462CB1838ACA2B02D9012003B000
:1013C000F0BD0023194600960822284601F092FC41
:1013D000731CD4B90822009311462346284601F015
:1013E00089FC10247378C82BE8D8012372785F1C1D
:1013F000013B934210D32B7FA88A0734E408B3B98A
:10140000844294BF00200120D9E7AB8ADB00083B6F
:10141000DB0873700824E5E7F319009321460023E5
:101420000822284601F066FC08343B46DEE7201A15
:1014300018BF0120C3E700002DE9F8430D4604461C
:101440001646002181222846FFF742FE2346082245
:101450000021284601F08AFDC6B9631C0722082135
:10146000284601F083FD0F2694F901306778002BA0
:10147000B8BF7F2704EB0709B0464C4508D10736B3
:10148000082010FB0760C008BDE8F8830826EBE7DA
:10149000A31C41460822284601F068FD08F108080F
:1014A0000134EAE72DE9F0410D46044616460021D5
:1014B000CE222846FFF70CFE23462822002128468C
:1014C00001F054FDBEB904F1080308222821284682
:1014D00001F04CFD302614F8080FC82828BFC8209A
:1014E00080460027B84506EBC70106D806EBC800C2
:1014F000C008BDE8F0812826EDE70137E31908228E
:10150000284601F033FDEDE7F7B5047F05460E46AA
:1015100034B1838AB3F5827F02D9012003B0F0BDD4
:101520000096012310220021284601F0E3FBDCB9DC
:10153000B31C0093092223461021284601F0DAFB50
:1015400019247388B3F5807FE7D837467288BB1BB0
:10155000934210D32B7FA88A0734E408B3B984429E
:1015600094BF00200120D9E7AB8ADB00103BDB08E9
:1015700073801024E5E73B1D0093214600230822D9
:10158000284601F0B7FB08340137DFE7201A18BFFF
:101590000120C3E730B5094D0A4491420DD011F83E
:1015A000013B5840082340F30004013B2C4013F05A
:1015B000FF0384EA5000F6D1EFE730BD2083B8ED99
:1015C000F7B54FF0FF33DFF854C0DFF854E000EB1D
:1015D00081011A4688421CD050F8044B019401AF97
:1015E000042417F8015B82EA05620825DB18164619
:1015F00005F1FF355241002EBCBF83EA0C0382EA9D
:101600000E0215F0FF05F1D1013C14F0FF04E8D102
:10161000E0E7D843D14303B0F0BD00BF9336EAA959
:10162000EBE1F042F7B5384A106851686B4603C3E6
:101630006A4636493648082302F056FF0446002819
:1016400033D10A25334A106851686B4603C36A4692
:1016500031492F48082302F047FF0446002849D0AB
:101660000369B3F5E02F45D8B0F8661041F2717206
:1016700091423FD1294A024402F15C018B4239D3A5
:101680005C3B234900209E1AFFF784FF3246074641
:1016900004F164010020FFF77DFFA3689F4229D178
:1016A000E368984208BF002524E00369B3F5E02F02
:1016B00027D8418B41F27172914220D1174A0244DE
:1016C00002F110018B4218D3103B114900209D1AE2
:1016D000FFF760FF2A46064604F118010020FFF7D5
:1016E00059FFA3689E4202D1E368984201D00D25BC
:1016F000A8E70025284603B0F0BD1025A2E70C2579
:10170000A0E70B259EE700BFD4450008DCFF0600DC
:1017100000000108DD45000890FF06000800FFF703
:1017200010B5037C044613B9006802F0C5FE2046DC
:1017300010BD00000023BFF35B8FC360BFF35B8F5E
:10174000BFF35B8F8360BFF35B8F7047BFF35B8F2B
:101750000068BFF35B8F704770B505460C30FFF72C
:10176000F5FF05F1080604463046FFF7EFFFA042FB
:1017700006D930466D68FFF7E9FF2544281A70BD89
:101780003046FFF7E3FF201AF9E7000070B5054681
:10179000406898B105F10800FFF7D8FF05F10C0685
:1017A00004463046FFF7D2FF8442304694BF6D684E
:1017B0000025FFF7CBFF013C2C44201A70BD000030
:1017C00038B50C460546FFF7C7FFA04210D305F118
:1017D0000800FFF7BBFF04446868B4FBF0F100FBAE
:1017E0001144BFF35B8F0120AC60BFF35B8F38BD4A
:1017F0000020FCE72DE9F041144607460D46FFF7AF
:10180000C5FF844228BF0446D4B1B84658F80C6BD3
:101810004046FFF79BFF3044286040467E68FFF754
:1018200095FF331A9C4203D86C600120BDE8F0811B
:101830006B60A41B3B68AB602044E8600220F5E7C6
:101840002046F3E738B50C460546FFF79FFFA04258
:1018500010D305F10C00FFF779FF04446868B4FB6E
:10186000F0F100FB1144BFF35B8F0120EC60BFF38C
:101870005B8F38BD0020FCE72DE9FF4188466946B3
:101880000746FFF7B7FF6C4606B204EBC606002515
:10189000B44209D06268206808EB0501FFF706FC36
:1018A000636808341D44F3E729463846FFF7CAFF4A
:1018B000284604B0BDE8F081F8B505460C300F4667
:1018C000FFF744FF05F1080604463046FFF73EFFE8
:1018D000A042304688BF6C68FFF738FF201A386096
:1018E00020B130462C68FFF731FF2044F8BD0000DE
:1018F00073B5144606460D46FFF72EFF844228BFF7
:1019000004460190DCB101A93046FFF7D5FF019BE9
:1019100033B93268C5E90233C5E9002401200CE07F
:101920009C4238BF01942860019868608442F5D9D0
:101930003368AB60241AEC60022002B070BD204610
:10194000FBE700002DE9FF410F466946FFF7D0FF96
:101950006C4600B204EBC0050026AC4209D0D4F8B6
:10196000048054F8081BB8194246FFF79FFB464411
:10197000F3E7304604B0BDE8F081000038B5054615
:10198000FFF7E0FF044601462846FFF719FF20460F
:1019900038BD000010B4026854681A4623465DF84A
:1019A000044B184700207047002070477047000024
:1019B000002070470E20704700F5805090F8C80056
:1019C000C0F340007047000000F5805090F9D0004F
:1019D0007047000000F58050C0F8CC10012070471F
:1019E000F7B50C68BDF8207014F0005470D10D7B71
:1019F000082D6DD8302585F311884569AE687601CC
:101A00000CD4AC68240108D4AC6814F080545DD1C7
:101A100084F31188204603B0F0BD01240E6804F160
:101A2000180C002EB8BFF6004FEA0C1CB4BF46F0ED
:101A30000406760545F80C600E680FFA84FC16F073
:101A4000804F18BF05EB0C1E05EB0C1C1EBFDEF80B
:101A5000806146F00206CEF880610E7BCCF884618E
:101A600005EB04158E68C5F88C614E68C5F8886171
:101A7000DCF8805145F00105CCF8805100EB4416AC
:101A800041F268052E4405EB44150544C6E90023E0
:101A900008350E4601F10C0C56F804EB45F804EB42
:101AA0006645F9D1843436882E8000EB441407F063
:101AB0000305267926F00B0635432571002484F3AF
:101AC0001188009700F0FCFC0120A4E70224A5E7A0
:101AD0004FF0FF309FE7000013B500F580540191EF
:101AE000E06DFFF753FE1F280AD90199E06D20220F
:101AF000FFF7C2FEA0F120035842584102B010BDCA
:101B00000020FBE708B5302383F3118800F58050EF
:101B1000C06DFFF70FFE002383F3118808BD00009E
:101B200000220260828142608260704710B500220C
:101B30000023C0E900230023044603810C30FFF793
:101B4000EFFF204610BD0000F0B5054600F58050BF
:101B50000C4690F8C83013F0040FC3F3800108BF9F
:101B6000114661F3820304F1840680F8C83005EB66
:101B7000461389B01B79D8072ED57AB319072DD40F
:101B80006846FFF7D3FF05EB441303F5835303F1D6
:101B9000180703AA103318685968144603C4083399
:101BA000BB422246F7D1186820609B88A380DDE9FC
:101BB0000E23CDE900230123ADF808302B686946D8
:101BC000DB6B2846984705EB46152B791A075CBF57
:101BD00043F008032B7101E0002AF4D109B0F0BDF5
:101BE0002DE9F0479A4688B007468846914630234B
:101BF00083F3118807F580546846FFF797FFE06D7F
:101C0000FFF7AAFD1F282AD9E06D20226946FFF7B9
:101C1000B5FE202823D103AD444605AB2E4603CEA6
:101C20009E4220606160354604F10804F6D13068B8
:101C30002060B388A380DDE90023C9E90023BDF853
:101C40000830AAF80030002383F3118853464A462F
:101C50004146384608B0BDE8F04700F01FBC002000
:101C600080F3118808B0BDE8F08700002DE9F84F37
:101C70000023C0E90133254B044640F8183B0F46CA
:101C8000FFF74EFF04F12800FFF750FF04F148086A
:101C900004F582554646083530462036FFF746FFA4
:101CA000AE42F9D104F580554FF480534FF000094E
:101CB000C5E91339C5F848800123EE6504F5875856
:101CC00004F58456C5F8549085F8583085F860308E
:101CD000083608F108084FF0000A4FF0000B46E9FB
:101CE00008ABA6F11800FFF71BFF203646F8289C2A
:101CF0004645F4D185F8D07017B1054800F0B8FB1F
:101D0000044B63612046BDE8F88F00BF1046000811
:101D1000E84500080064004010B5044B19780446FB
:101D20004A1C1A70FFF7A2FF204610BD1C4A002073
:101D30002DE9F047002950D0294B2A4FB7FBF1F588
:101D400099428CBF0A231123581EB5FBF3FC03FBF9
:101D50001C53C4B22BB102280346F5D80020BDE8BD
:101D6000F0870CF1FF36B6F5806FF7D2C4EBC40EE6
:101D70000EF103034FEAE309C3F3C703A4EB03081F
:101D800009F1010A4FF47A755FFA88F009FB0555ED
:101D90005AFA88F8B5FBF8F5B5F5617FC1BF0EF1C9
:101DA000FF33C3F3C703E01AC0B25C1C50FA84F4DB
:101DB0000CFB04F4B7FBF4F4A142CFD1013BDBB23E
:101DC0000F2BCBD80138C0B20728C7D8002110711B
:101DD00016809170D3700120C1E70846BFE700BFAD
:101DE0003F420F0080DE800270B505460E464FF47C
:101DF0007A746B695B6803F00103B34207D04FF458
:101E00007A7001F095FC013CF3D1204670BD0120B1
:101E1000FCE7000030B54269936913F0700F16D0EB
:101E200000230B4C936103F1840200EB4212117901
:101E30004D0709D5890707D5416954F823508D60AE
:101E4000117941F0040111710133032BEBD130BD45
:101E5000FC45000873B51D46436916469A68D207CB
:101E6000044609D59A6801219960C2F34002CDE980
:101E700000650021FFF768FE63699A68D1050BD5FC
:101E80009A684FF480719960C2F34022CDE90065F1
:101E900001212046FFF758FE63699A68D2030BD5EB
:101EA0009A684FF480319960C2F34042CDE90065F1
:101EB00002212046FFF748FE04F58053D3F8CC00FA
:101EC00010B103681B699847204602B0BDE8704016
:101ED000FFF7A0BFF8B504464669002972D106F1A4
:101EE0000C073868800770D006EB01153868D5F804
:101EF000B00110F0040FD5F8B0011ABFC00840F0CF
:101F00000040400DA061D5F8B0C11CF0020F1CBF0D
:101F100040F08040A061D5F8B40106EB011100F05B
:101F20000F0084F82400D1F8B8012077D1F8B80167
:101F3000000A6077D1F8B801000CA077D1F8B80199
:101F4000000EE077D1F8BC0184F82000D1F8BC0184
:101F5000000A84F82100D1F8BC01000C84F82200AA
:101F6000D1F8BC11090E84F823103821396004F12E
:101F7000340004F1180104F1240551F8046B40F811
:101F8000046BA942F9D109880180C4E90A232146DA
:101F90000023238651F8283B2046DB6B984704F545
:101FA000805393F8C820D3F8CC0042F0040283F8A1
:101FB000C82010B103681B6998472046BDE8F84067
:101FC000FFF728BF06F110078BE7F8BD10B50446F0
:101FD00000F056FA02460B4652EA030102D0013ADB
:101FE00063F100030449086820B12146BDE81040B0
:101FF000FFF770BF10BD00BF184A0020F0B53021B8
:1020000081F31188DFF848C000F5835108310024BE
:1020100004F1840500EB45152E7977070ED4F606FA
:102020000CD5D1E9007697429E4107D246695CF80B
:102030002470B7602E7946F004062E710134032C0B
:1020400001F12001E4D1002383F31188F0BD00BF2A
:10205000FC45000808B5302383F31188FFF7DAFE4A
:10206000002383F3118808BDF8B5436905469868D5
:1020700000F0E050B0F1E05F0F4621D0F8B130231E
:1020800083F3118805F583541034002606F1840388
:1020900005EB43131B791A0706D50136032E04F10D
:1020A0002004F3D1012007E05B07F6D4214638462F
:1020B00000F040FA0028F0D1002383F31188F8BD26
:1020C0000120FCE708B5302383F3118800F5805028
:1020D000C06DFFF741FB002383F3118843090CBF58
:1020E0000120002008BD0000F8B51D460023137034
:1020F0000F4606461446FFF7E5FF80F001003870F2
:1021000025B129463046FFF7AFFF2070F8BD00002B
:102110002DE9B8410C4615461F46804600F0B0F93F
:102120000B462178024609B9287850B14046FFF79E
:1021300065FFFFF78FFF3B462A462146FFF7D4FF96
:102140000120BDE8B881000070B5302686F3118803
:10215000174B1A6C42F000721A641A6A42F000724D
:102160001A621A6A22F000721A62002383F311883D
:1021700000F5805494F8C83013F0010516D1A9B1C8
:1021800086F311880321132001F0CEF903211420D6
:1021900001F0CAF90321152001F0C6F994F8C830FE
:1021A00043F0010384F8C83085F3118870BD00BF87
:1021B000003802402DE9F04700F5805588B095F8C9
:1021C000D030012B04468846164600F28180814FAC
:1021D00057F823200AB947F82300D7F800A0C4F81D
:1021E0000C802674BAF1000F64D095F8D030012B22
:1021F00070D001212046FFF7A7FF302383F3118819
:102200006269136823F0020313606269136843F084
:1022100001031360636900275F6187F3118801215F
:102220002046FFF7E1FD002800F09580E86DFFF7FC
:1022300081FA04F58359BA4609F1080920220021E0
:102240006846FEF745FF02A8FFF76AFCCDF818A024
:102250006A4609EB07030DF1180E9446BCE803002B
:10226000F44518605960624603F10803F5D1DCF8C3
:102270000000186020379CF804201A71602FDDD10F
:1022800095F8C8306FF38203002785F8C8306A4696
:1022900041462046ADF80070ADF802708DF804702C
:1022A000FFF746FD636948BB4FF400421A6008B06F
:1022B000BDE8F08741F2D80002F0BEF8814610B1C7
:1022C0005146FFF7D3FCC7F80090B9F1000F8CD14D
:1022D0000020ECE7386803681B6B9847014600282C
:1022E00087D13868FFF730FF3868036832465B688B
:1022F0004146984700287FF47CAFE9E761221A60E5
:102300009DF802309DF803201B06120402F470228F
:1023100003F040731343BDF80020C2F309021343D6
:102320009DF804201205022E02F4E0020CBF4FF0CB
:1023300000410021134362690B43D3616369132297
:102340005A616269136823F001031360394620461D
:10235000FFF74AFD08B96369A6E795F8D03093BB4B
:102360006169D1F8002242F00102C1F800226169DE
:10237000D1F8002222F47C5222F00E02C1F8002291
:102380006169D1F8002242F46062C1F800226269FA
:10239000C2F814326269C2F80432626941F6FF7110
:1023A000C2F80C126269C2F840326269C2F8443263
:1023B00063690122C3F81C226269D2F8003223F05B
:1023C0000103C2F8003295F8C83043F0020385F8E3
:1023D000C8306CE7184A002008B500F051F850EA00
:1023E0000103024602D0421E61F10001044B18684D
:1023F00010B10B46FFF72EFDBDE8084001F06AB8AA
:10240000184A002008B50020FFF7E0FDBDE80840AD
:1024100001F060B808B50120FFF7D8FDBDE808401D
:1024200001F058B800B59BB0EFF309816822684607
:10243000FEF73CFEEFF30583014B9B6BFEE700BF0D
:1024400000ED00E008B5FFF7EDFF000000B59BB020
:10245000EFF3098168226846FEF728FEEFF3058353
:10246000014B5B6BFEE700BF00ED00E0FEE7000004
:102470000FB408B5029801F00BF9FEE701F00EBCAD
:1024800001F0F0BB13B56C4684E80600031D94E828
:10249000030083E80500012002B010BD73B5856814
:1024A000019155B11B885B0707D4D0E900369B6BBF
:1024B0009847019AC1B23046A847012002B070BDCA
:1024C000F0B5866889B005460C465EB1BDF8383077
:1024D0005B070AD4D0E900379B6B98472246C1B20C
:1024E0003846B047012009B0F0BD00220023CDE9F5
:1024F00000230023ADF808300A4603AB01F10806BB
:10250000106851681C4603C40832B2422346F7D112
:10251000106820609288A280FFF7B2FF0423ADF814
:1025200008302B68CDE90001DB6B694628469847E7
:10253000D8E7000030B503680968DD0FB5EBD17F3F
:1025400023F0604421F060424FEAD1700BD0002BA1
:10255000B8BFA40C0029B8BF920C944202D034BF7B
:102560000120002030BD944205D1C1F38070C3F337
:1025700080738342F6D194422CBF00200120F1E702
:102580002DE9F041456A15B94162BDE8F0814B681B
:1025900023F06047C3F38A464FEAD37EC3F38078C3
:1025A00016EA230638BF3E46AC462B465A68BEEBB9
:1025B000D27F22F060440AD0002A18DAA40CB44278
:1025C00017D19D420FD10D60DEE71346EEE7A7421B
:1025D00007D102F08044C2F3807242450BD054B15F
:1025E000EFE708D2EDE7CCF800100B60CDE7B4427E
:1025F00001D0B442E5D81A689C46002AE5D119609A
:10260000C3E700002DE9F047089D01F007044FEAF9
:10261000D508224405F0070500EBD1004FF47F49AF
:10262000944201D1BDE8F08704F0070705F0070ADE
:1026300057453E4638BF5646C6F10806111B8E4226
:1026400028BF0E46E10808EBD50E415C13F80EC01A
:10265000B94029FA06F721FA0AF1FFB28CEA010122
:1026600047FA0AF739408CEA010C03F80EC03444EB
:102670003544D5E780EA0120082341F2210201B266
:102680004000002980B203F1FF33B8BF504013F07F
:10269000FF03F4D17047000038B50C468D18A542F1
:1026A00000D138BD14F8011BFFF7E4FFF7E7000085
:1026B00042684AB1136843604389818901339BB200
:1026C0009942438138BF83811046704770B588B006
:1026D000202204460D4668460021FEF7F9FC2046FC
:1026E0000495FFF7E5FF024658B16B46054608AE74
:1026F0001C4603CCB44228606960234605F10805F6
:10270000F6D1104608B070BD082817D909280CD09A
:102710000A280CD00B280CD00C280CD00D280CD07B
:102720000E2814BF4020302070470C207047102026
:102730007047142070471820704720207047000011
:10274000082817D90C280CD910280CD914280CD912
:1027500018280CD920280CD930288CBF0F200E2027
:102760007047092070470A2070470B2070470C20E3
:1027700070470D20704700002DE9F843078C072FA4
:1027800004461ED9D0E9029800254FF6FF73C5F123
:102790002006A5F1200029FA05F108FA06F628FA24
:1027A00000F031430143C9B21846FFF763FF083513
:1027B000402D0346EBD1E1693A46BDE8F843FFF707
:1027C0006BBF4FF6FF70BDE8F883000010B54B6893
:1027D00023B9CA8A63F30902CA8210BD04691A6860
:1027E0001C600361C38A013BC3824A60EFE70000BB
:1027F0002DE9F84F1D46CB8A0F46C3F30901052981
:10280000814692460B4630D00020AAB207F11A0446
:102810009EB2042E1FFA80F80FD8904503F10103F1
:1028200006D3FB8A0A4462F30903FB8201201AE003
:102830001AF80060E6540130EAE79045F1D2A1F1C0
:10284000050B1C237C68BBFBF3F203FB12BB1FFAD6
:102850008BF6002C45D14846FFF72AFF044638B9CD
:1028600078606FF00200BDE8F88F4FF00008E6E7EF
:10287000002606607860ADB24FF0000B454510D9D8
:102880000AEB0803221D13F8011B9155B1B208F1A0
:1028900001081B291FFA88F82BD0454506F10106CF
:1028A000F1D8FB8AC3F30902154465F30903BCE7B9
:1028B000013292B21C462368002BF9D16B1F0B44E6
:1028C0001C21B3FBF1F301339BB29A42D3D2BBF18B
:1028D000000FD0D14846FFF7EBFE20B9C4F800B096
:1028E000BFE70122E7E7C0F800B05E46206004467B
:1028F000C1E74545D5D94846FFF7DAFE08B920605B
:10290000AFE7C0F800B0002620600446B6E700003C
:102910002DE9F04F2DED028B1C4683B05B690192CF
:1029200007468846002B00F09A80238C2BB1E26981
:10293000002A00F09480072B35D807F10C00FFF730
:10294000B7FE054638B96FF00205284603B0BDEC66
:10295000028BBDE8F08F14220021FEF7B9FB228C18
:10296000E16905F10800FEF7A1FB208C013080B27F
:10297000FFF7E6FEFFF7C8FE013880B22084013081
:1029800028746369228C1B782A4403F01F0363F0C8
:102990003F0348F000411372384669602946FFF74B
:1029A000EFFD0125D1E700F10C034FF0000908EE1F
:1029B000103A4FF0800A4E464D4618EE100AFFF7C7
:1029C00077FE83460028BED014220021FEF780FB4C
:1029D000002E3AD1019BABF8083002220BF1080E11
:1029E0001FFA82FC0CF10100BCF1060F218C80B2B1
:1029F00001D88E422BD3FFF7A3FEFFF785FE626955
:102A00001278013802F01F028E4208BF4FF0400AD0
:102A100042EA49121BFA80F14AEA020A013048F000
:102A2000004281F808A08BF81000CBF8042059462A
:102A30003846FFF7A5FD238C0135B3422DB289F04E
:102A400001094FF0000AB8D17FE70022C6E7E1692B
:102A5000895D0EF802100136B6B20132C0E76FF0A0
:102A6000010572E7F8B515460E46302200210446EE
:102A70001F46FEF72DFB069B6360B5F5001F079B05
:102A8000A76034BF6A094FF6FF72A36297B2E6618E
:102A900004F1100000239A4206D800230360A782A5
:102AA000E3822383E360F8BD0660013330462036BD
:102AB000F1E7000003781BB94BB2002BC8BF0170CF
:102AC0007047000000787047F8B50C46C9690746A2
:102AD00011B9238C002B37D1257E1F2D34D838789F
:102AE00028BB228C072A2CD8268A36F003032BD148
:102AF0004FF6FF70FFF7D0FD20F0010031024004D7
:102B000041EA0561400C41EA40254FF6FF72234639
:102B100029463846FFF7FCFE002807DD6269137876
:102B20000133DBB21F2B88BF00231370F8BD218A4D
:102B30002D0645EA012505432046FFF71DFE024606
:102B4000E5E76FF00300F1E76FF00100EEE700004A
:102B500070B58AB0044616460021282268461D46F4
:102B6000FEF7B6FABDF83830ADF810300F9B05937C
:102B70009DF840308DF81830119B07936946BDF8D9
:102B80004830ADF820302046CDE90265FFF79CFFC4
:102B90000AB070BD2DE9F041D36905460C461646D2
:102BA0000BB9138C5BBB377E1F2F28D895F800809C
:102BB000B8F1000F26D03046FFF7DEFD3378210252
:102BC00041EAC33141EA0801338A41EA076141EA37
:102BD00003410246334641F080012846FFF798FE44
:102BE00000280ADD3378012B07D17269137801338D
:102BF000DBB21F2B88BF00231370BDE8F0816FF09C
:102C00000100FAE76FF00300F7E70000F0B58BB0C2
:102C100004460D4617460021282268461E46FEF748
:102C200057FA9DF84C305A1E534253418DF80030EC
:102C30009DF84030ADF81030119B05939DF8483059
:102C40008DF81830149B07936A46BDF85430ADF8E0
:102C5000203029462046CDE90276FFF79BFF0BB0D6
:102C6000F0BD0000406A00B104307047436A1A6842
:102C7000426202691A600361C38A013BC3827047E2
:102C80002DE9F041D0F82080194E14461D464146EA
:102C9000002709B9BDE8F081D1E90223A21A65EB4A
:102CA0000303964277EB03031ED2036A8B420DD1D6
:102CB000FFF78CFD036A1B68036203690B60C38A1C
:102CC0000161016A013BC3828846E2E7FFF77EFDAE
:102CD0000B68C8F8003003690B60C38A0161013BCF
:102CE000C382D8F80010D4E788460968D1E700BF4E
:102CF00080841E002DE9F04F8BB00D46DDF850901A
:102D000014469B468046002800F01981B9F1000F57
:102D100000F01581531E3F2B00F21181012A03D1CF
:102D2000BBF1000F40F00B810023CDE90833B8F868
:102D30001430B5EBC30F4FEAC30703D300200BB029
:102D4000BDE8F08F2B199F42D8F80C303ABF7F1B9B
:102D5000FFB227461BB9D8F81030002B7AD0272DA8
:102D60004ED8C5F12806B7424FF000032CBFF6B28B
:102D70003E4600932946D8F8080008AB3246FFF7D4
:102D800041FCA7EB060A35445FFA8AFAB8F814301A
:102D900003F10053053BDB000493D8F80C30039398
:102DA0002821039B13B1BAF1000F2CD1D8F81000E1
:102DB00040B1BAF1000F05D0009608AB5246691A2F
:102DC000FFF720FC38B2002FB8D066070AD00AAB54
:102DD00003EBD401624211F8083C02F007021341F0
:102DE00001F8083C082C3CD9102C40F2B580202C6E
:102DF00040F2B780BBF1000F00F09C80082334E064
:102E0000BA460026C2E7049BE02B28BFE0230693C6
:102E10000B44AB42059314D95A1B03980096924574
:102E200034BF5246D2B2691A08AB04300792FFF79A
:102E3000E9FB079A1644AAEB020A1544F6B25FFAB8
:102E40008AFA049B069A05999B1A0493039B1B68B4
:102E50000393A6E70093D8F8080008AB3A46294642
:102E6000AEE7BBF1000F13D00123B4EBC30F6CD05E
:102E7000082C12D89DF82030621E23FA02F2D507E2
:102E800006D54FF0FF3202FA04F423438DF82030C8
:102E90009DF8203089F8003051E7102C12D8BDF889
:102EA0002030621E23FA02F2D10706D54FF0FF321E
:102EB00002FA04F42343ADF82030BDF82030A9F81D
:102EC00000303CE7202C0FD80899631E21FA03F349
:102ED000DA0705D54FF0FF3202FA04F40C430894E8
:102EE000089BC9F800302AE7402C2BD0DDE90865A3
:102EF000611EC4F12102A4F1210326FA01F105FAB1
:102F000002F225FA03F311431943CB0712D501222C
:102F1000A4F12003C4F1200102FA03F322FA01F123
:102F2000A240524243EA010363EB430332432B4383
:102F3000CDE90823DDE90823C9E90023FFE66FF0A6
:102F40000100FCE66FF00800F9E6082CA0D9102C6F
:102F5000B3D9202CEED8C3E7BBF1000FADD00223CC
:102F600083E7BBF1000FBBD004237EE730B5012A15
:102F7000144638BF0124402C85B028BF40240025CA
:102F8000012ACDE9025518D81B788DF8083063075F
:102F90000AD004AB03EBD405624215F8083C02F0FA
:102FA0000702934005F8083C0091034622460021A1
:102FB00002A8FFF727FB05B030BD082AE4D9102A84
:102FC00003D81B88ADF80830E1E7202A8DBFD3E98C
:102FD00000231B680293CDE90223D8E710B5CB6824
:102FE0001BB98B600B618B8210BD04691A681C6071
:102FF0000361C38A013BC382CA60F0E703064CBF8A
:10300000C0F3C0300220704708B50246FFF7F6FF54
:10301000022806D15306C2F30F2001D100F00300AD
:1030200008BDC2F30740FBE72DE9F04F93B0CDE9AF
:1030300003230A6804461046FFF7E0FF022814BF86
:10304000C2F306260026002A0D46824680F2F7814A
:1030500012F0C04940F0F381097B002900F0EF81B4
:10306000022803D02378B34240F0EC81C2F304631A
:103070000693104602F07F030593FFF7C5FF059BFB
:1030800029444FEA834848EA0A4848EA4668CE7825
:1030900000230022CDE90823F309834648EA00080B
:1030A000029367D0059B009302466768534608A9C0
:1030B0002046B847002800F0C881276A4FB941462A
:1030C00004F10C00FFF702FB074690B96FF0020015
:1030D00054E03B6998450DD03F68002FF9D1414637
:1030E00004F10C00FFF7F2FA07460028EED0236A3D
:1030F0003B60276297F817C006F01F08CCF3840CDA
:10310000ACEB08001FFA80FE0028B8BF0EF12000CB
:10311000A8EB0C031FFA83FED7E90221B8BF00B267
:10312000002B0793BEBF0EF120031BB2079352EA98
:10313000010338D0039BDFF824E39A1A049B4FF075
:10314000000C63EB010196457CEB01032BD36B7BF9
:1031500097F81AE0734519D1029B002B78D001280B
:1031600021DC7868F8B9DFF8F0C2944570EB010310
:1031700016D337E0276A27B96FF00C0013B0BDE80B
:10318000F08F3B699845B5D03F68F4E7B24890426C
:103190007CEB010301D30020F0E7029B002BFAD067
:1031A000079B0F2B17DCFA7DB30002F0030203F03C
:1031B0007C031343FB7539462046FFF707FB6B7B07
:1031C000BB76029B3BB9FB7DC3F38402013262F301
:1031D0008603FB75D0E76A7BBB7E9A42DBD1029BFC
:1031E000002B35D0B309022B32D0039BBB60049B6C
:1031F000FB60142200210DA8FDF76AFF039B0A93D0
:10320000049B0B932B1D0C932B7BADF83EB0013B25
:10321000DBB2ADF83C30069B8DF84230059B8DF853
:10322000433094F82C308DF840A083F001038DF8E2
:1032300044308DF84180A3680AA920469847FB7D59
:10324000C3F38403013303F01F039B02FB82A2E755
:10325000FB7DC6F34012B2EBD31F40F0F980C3F3FD
:103260008403434540F0FC80029A2B7BB609002A78
:1032700052D016F0010661D1032B40F2F480039B7B
:10328000BB60049BFB60FB8A66F30903FB822B7B1C
:10329000AE1D033BDBB23246394604F10C00FFF7AA
:1032A000A7FA00280CDA39462046FFF78FFAFB7D93
:1032B000C3F38403013303F01F039B02FB8205E782
:1032C000DDE90884AB883B834FF6FF73C9F120002A
:1032D000A9F1200228FA09F104FA00F0014324FAC6
:1032E00002F211431846C9B2FFF7C4F909F10809FF
:1032F000B9F1400F0346E9D1B8822A7B033AD2B232
:103300003146FFF7C9F9FB7DB882DA43C2F3C01238
:1033100062F3C713FB753EE786B92E1D013BDBB296
:103320003246394604F10C00FFF762FA0028BADB96
:103330002A7BB88A013AD2B23146E2E7F98AC1F370
:103340000901013B0429DAB25BD8281D002307F1EB
:103350001B069A4208D910F801CB06F801C00131CA
:1033600001330529DBB2F4D103990A9104990B9139
:10337000934207F11B010C9138BF043379680D911A
:1033800034BF55FA83F300230E93FB8AADF83EB0A9
:10339000C3F309031A44069B8DF84230059B8DF850
:1033A000433094F82C30ADF83C2083F001038DF8C5
:1033B000443000238DF840A08DF841807B602A7B4B
:1033C000B88A013A291DFFF767F93B8BB88283421F
:1033D00003D1A3680AA92046984720460AA9FFF707
:1033E000FDFDFB7DBA8AC3F38403013303F01F03A1
:1033F0009B02FB823B8B9A420CBF00206FF01000B7
:10340000BCE67B68002BAFD0052001E01C303346C2
:103410001E68002EFAD1091A081D2E1D184401EB52
:10342000090CBCF11B0F5FFA89F39DD89A429BD916
:1034300016F8013B00F8013B09F10109EFE76FF0D5
:1034400009009BE66FF00A0098E66FF00B0095E626
:103450006FF00D0092E600BF40420F0080841E0016
:103460006FF00E008AE66FF00F0087E6EFF3098336
:1034700005494A6B22F001024A63683383F30988E5
:10348000002383F31188704700EF00E0302080F3C1
:10349000118862B60C4B0D4AD96821F4E061090429
:1034A000090C0A43DA60D3F8FC20094942F0807223
:1034B000C3F8FC200A6842F001020A602022DA7791
:1034C00083F82200704700BF00ED00E00003FA051A
:1034D000001000E010B5302383F311880E4B5B68B9
:1034E00013F4006314D0F1EE103AEFF30984683C52
:1034F0004FF08073E361094BDB6B236684F309882B
:1035000000F090F810B1064BA36110BD054BFBE72E
:1035100083F31188F9E700BF00ED00E000EF00E061
:103520003F0300084203000800F1604303F56143D4
:103530000901C9B283F80013012200F01F039A4069
:1035400043099B0003F1604303F56143C3F8802105
:103550001A60704700230375826803691B689968C5
:103560009142FBD25A680360426010605860704715
:1035700000230375826803691B6899689142FBD830
:103580005A680360426010605860704708B508468A
:10359000302383F311880B7D032B05D0042B0DD032
:1035A0002BB983F3118808BD8B6900221A604FF094
:1035B000FF338361FFF7CEFF0023F2E7D1E900324A
:1035C00013605A60F3E70000FFF7C4BF054BD968EA
:1035D0000875186802681A60536001220275D86085
:1035E000FCF798BE284A002030B50C4BDD684B1C18
:1035F00087B004460FD02B46094A684600F02AF9E6
:103600002046FFF7E3FF009B13B1684600F02CF95A
:10361000A86907B030BDFFF7D9FFF9E7284A0020B5
:103620008D350008044B1A68DB6890689B689842E7
:1036300094BF002001207047284A0020084B10B595
:103640001C68D86822681A60536001222275DC6009
:10365000FFF78EFF01462046BDE81040FCF75ABE3A
:10366000284A002038B5074C07490848012300259F
:103670002370656000F016FC0223237085F3118827
:1036800038BD00BF904C002054460008284A002056
:1036900008B572B6044B186500F0C6FA00F07CFB62
:1036A000024B03221A70FEE7284A0020904C0020AB
:1036B00000F010B98B60022308618B8208467047C6
:1036C0008368A3F1840243F8142C026943F8442C64
:1036D000426943F8402C094A43F8242CC26843F855
:1036E000182C022203F80C2C002203F80B2C044A9D
:1036F00043F8102CA3F12000704700BF2D030008F1
:10370000284A002008B5FFF7DBFFBDE80840FFF7B7
:103710005BBF0000024BDB6898610F20FFF756BFCC
:10372000284A0020302383F31188FFF7F3BF0000FD
:1037300008B50146302383F311880820FFF754FFB2
:10374000002383F3118808BD10B503689C68A2426A
:103750000CD85C688A600B604C6021605960996885
:103760008A1A9A604FF0FF33836010BD1B68121BEA
:10377000ECE700000A2938BF0A2170B504460D465F
:103780000A26601900F088FB00F074FB041BA542B8
:1037900003D8751C2E460446F3E70A2E04D9BDE86B
:1037A0007040012000F0BEBB70BD0000F8B5144BA6
:1037B0000D46D96103F1100141600A2A196982603E
:1037C00038BF0A22016048601861A818144600F04A
:1037D00055FB0A2700F04EFB431BA342064606D3C7
:1037E0007C1C281900F058FB27463546F2E70A2FC3
:1037F00004D9BDE8F840012000F094BBF8BD00BF3B
:10380000284A0020F8B506460D4600F033FB0F4A63
:10381000134653F8107F9F4206D12A460146304690
:10382000BDE8F840FFF7C2BFD169BB68441A2C1944
:1038300028BF2C46A34202D92946FFF79BFF224608
:1038400031460348BDE8F840FFF77EBF284A002014
:10385000384A002010B4C0E9032300235DF8044B6C
:103860004361FFF7CFBF000010B5194C23699842A0
:103870000DD0D0E90032816813605A609A680A441A
:103880009A60002303604FF0FF33A36110BD23460D
:10389000026843F8102F53600022026022699A42A6
:1038A00003D1BDE8104000F0F1BA936881680B4481
:1038B000936000F0DFFA2269E1699268441AA2423B
:1038C000E4D91144BDE81040091AFFF753BF00BF07
:1038D000284A00202DE9F047DFF8BC8008F11007E6
:1038E0002C4ED8F8105000F0C5FAD8F81C40AA6841
:1038F000031B9A423ED81444D5E900324FF0000928
:10390000C8F81C4013605A60C5F80090D8F8103011
:10391000B34201D100F0BAFA89F31188D5E9033135
:1039200028469847302383F311886B69002BD8D041
:1039300000F0A0FA6A69A0EB04094A4582460DD25C
:10394000022000F0EFFA0022D8F81030B34208D17C
:1039500051462846BDE8F047FFF728BF121A224417
:10396000F2E712EB090938BF4A4629463846FFF705
:10397000EBFEB5E7D8F81030B34208D01444211A52
:10398000C8F81C00A960BDE8F047FFF7F3BEBDE82A
:10399000F08700BF384A0020284A002038B500F0E0
:1039A00069FA054AD2E90845031B181945F10001D7
:1039B000C2E9080138BD00BF284A00200020704736
:1039C000FEE70000704700004FF0FF307047000036
:1039D000BFF34F8F024AD368DB03FCD4704700BFAC
:1039E000003C024008B5094B1B7873B9FFF7F0FFA4
:1039F000074B1A69002ABFBF064A5A6002F1883293
:103A00005A601A6822F480621A6008BD984C00203F
:103A1000003C02402301674508B50B4B1B7893B966
:103A2000FFF7D6FF094B1A6942F000421A611A6883
:103A300042F480521A601A6822F480521A601A689E
:103A400042F480621A6008BD984C0020003C02409D
:103A50000728F0B516D80C4C0C4923787BB90C4DCF
:103A60000E4608234FF0006255F8047B46F8042BFD
:103A7000013B13F0FF033A44F6D10123237051F8C0
:103A80002000F0BD0020FCE7BC4C00209C4C002036
:103A900060460008014B53F820007047604600085C
:103AA00008207047072810B5044601D9002010BD32
:103AB000FFF7CEFF064B53F824301844C21A0BB957
:103AC0000120F4E712680132F0D1043BF6E700BFB1
:103AD00060460008072810B5044621D8FFF778FF94
:103AE000FFF780FF0F4AF323D360C300DBB243F438
:103AF000007343F002031361136943F480331361CD
:103B0000FFF766FFFFF7A4FF074B53F8241000F000
:103B10003FF9FFF781FF2046BDE81040FFF7C2BF25
:103B2000002010BD003C024060460008F8B512F0CD
:103B30000103144642D185182E4A954257D82E4B80
:103B40001B6813F0010352D02C4DFFF74BFFF323FA
:103B5000EB60FFF73DFF40F20127032C15D824F05E
:103B600001046618254C401A40F20117B14223693E
:103B700000EB010524D123F001032361FFF74CFF83
:103B80000120F8BD043C0430E7E78307E7D12B6947
:103B900023F440732B612B693B432B6151F8046B79
:103BA0000660BFF34F8FFFF713FF03689E42E9D013
:103BB0002B6923F001032B61FFF72EFF0020E0E7C4
:103BC00023F44073236123693B4323610B882B80DB
:103BD000BFF34F8FFFF7FCFE2D8831F8023BADB2EB
:103BE000AB42C3D0236923F001032361E4E7184605
:103BF000C7E700BF0000080800380240003C024050
:103C0000084908B50B7828B11BB9FFF7EBFE012373
:103C10000B7008BD002BFCD0BDE808400870FFF712
:103C2000FBBE00BF984C002008B50649064800F0CE
:103C3000B1F8BDE808404FF480314FF0805000F0FB
:103C4000A9B800BF00FF010000010020084611468E
:103C500000F014BC012000F011BC0000084600F088
:103C60002BBC000038B5EFF311859DB9EFF3058447
:103C7000C4F30804302334B183F31188FFF78EFEB8
:103C800085F3118838BD83F31188FFF787FE84F32D
:103C9000118838BDBDE83840FFF780BE38B5FFF762
:103CA000E1FF114C114AC00840EA4170A0FB025EDE
:103CB000C908A0FB040C1CEB050CA1FB04404FF051
:103CC00000035B41A1FB02121CEB040C43EB000060
:103CD00011EB0E0142F10002411842F10000090906
:103CE00041EA007038BD00BFCFF753E3A59BC42065
:103CF00010B50244064BD2B2904200D110BD441C14
:103D000000B253F8200041F8040BE0B2F4E700BF22
:103D1000502800400F4B30B51C6F240407D41C6F93
:103D200044F400741C671C6F44F400441C670A4C84
:103D3000236843F4807323600244084BD2B290425C
:103D400000D130BD441C00B251F8045B43F8205050
:103D5000E0B2F4E700380240007000405028004014
:103D600007B5012201A90020FFF7C2FF019803B0A7
:103D70005DF804FB13B50446FFF7F2FFA04205D03F
:103D8000012201A900200194FFF7C4FF02B010BD79
:103D9000704700007047000070470000074B45F275
:103DA00055521A6002225A6040F6FF729A604CF631
:103DB000CC421A60024B01221A707047003000405A
:103DC000C44C0020034B1B781BB1034B4AF6AA22BC
:103DD0001A607047C44C002000300040034B1A6842
:103DE0001AB9034AD2F874281A607047C04C0020F0
:103DF00000300240024B4FF08072C3F874287047C5
:103E00000030024008B5FFF7E9FF024B1868C0F325
:103E1000407008BDC04C002008B5FFF7DFFF024B23
:103E20001868C0F3007008BDC04C00207047000047
:103E3000FEE700000A4B0B480B4A90420BD30B4B9A
:103E4000DA1C121AC11E22F003028B4238BF002274
:103E50000021FDF73DB953F8041B40F8041BECE7C3
:103E600008480008504D0020504D0020504D0020C3
:103E700000F0D0B84FF08043586A70474FF080434D
:103E8000002258631A610222DA6070474FF08043C3
:103E90000022DA60704700004FF08043586370479B
:103EA000FEE7000070B51B4B01630025044686B099
:103EB000586085620E46FFF7E9FA04F11003C4E981
:103EC00004334FF0FF33C4E90635C4E90044A5606C
:103ED000E562FFF7CFFF2B460246C4E9082304F151
:103EE00034010D4A256580232046FFF7E3FB0123BB
:103EF000E0600A4A0375009272680192B268CDE9E7
:103F00000223074B6846CDE90435FFF7FBFB06B0FB
:103F100070BD00BF904C0020804600088546000818
:103F2000A13E0008024AD36A1843D062704700BF1E
:103F3000284A00204B6843608B688360CB68C3606D
:103F40000B6943614B6903628B6943620B680360D1
:103F50007047000008B5264B26481A6940F2FF1149
:103F60000A431A611A6922F4FF7222F001021A61EF
:103F70001A691A6B0A431A631A6D0A431A651E4AB4
:103F80001B6D1146FFF7D6FF02F11C0100F58060A2
:103F9000FFF7D0FF02F1380100F58060FFF7CAFF9C
:103FA00002F1540100F58060FFF7C4FF02F17001D7
:103FB00000F58060FFF7BEFF02F18C0100F5806024
:103FC000FFF7B8FF02F1A80100F58060FFF7B2FF2C
:103FD00002F1C40100F58060FFF7ACFF02F1E001DF
:103FE00000F58060FFF7A6FFBDE8084000F08EB83E
:103FF00000380240000002408C46000808B500F07E
:10400000F9F9FFF72FFBBDE80840FFF7E7BE000016
:10401000704700000F4B1A6C42F001021A641A6ECE
:1040200042F001021A660C4A1B6E936843F00103CA
:1040300093604FF0804353229A624FF0FF32DA626E
:1040400000229A615A63DA605A6001225A611A604A
:10405000704700BF00380240002004E04FF080426B
:1040600008B51169D3680B40D9B2C9439B071161E8
:1040700007D5302383F31188FFF71AFB002383F35E
:10408000118808BD1F4B1A696FEAC2526FEAD252FB
:104090001A611A69C2F308021A614FF0FF301A69F7
:1040A0005A69586100215A6959615A691A6A62F05D
:1040B00080521A621A6A02F080521A621A6A5A6AA6
:1040C00058625A6A59625A6A1A6C42F080521A64EB
:1040D0001A6E42F080521A661A6E0B4A106840F44B
:1040E00080701060186F00F44070B0F5007F1EBF44
:1040F0004FF4803018671967536823F400735360D6
:1041000000F054B90038024000700040334B4FF0CB
:1041100080521A64324A4FF4404111601A6842F0EA
:1041200001021A601A689107FCD59A6822F003020E
:104130009A602A4B9A6812F00C02FBD1196801F0C0
:10414000F90119609A601A6842F480321A601A689C
:104150009203FCD55A6F42F001025A671F4B5A6F07
:104160009007FCD51F4A5A601A6842F080721A60A4
:104170001B4A53685904FCD5184B1A689201FCD5A8
:10418000194A9A60194B1A68194B9A42194B21D156
:10419000194A1168194A91421CD140F205121A605D
:1041A000144A136803F00F03052BFAD10B4B9A68DE
:1041B00042F002029A609A6802F00C02082AFAD1D0
:1041C0005A6C42F480425A645A6E42F480425A66F3
:1041D0005B6E704740F20572E1E700BF00380240B5
:1041E000007000400854400700948838002004E024
:1041F00011640020003C024000ED00E041C20F418C
:10420000074A08B5536903F00103536123B1054A16
:1042100013680BB150689847BDE80840FFF75AB9DA
:10422000003C0140C84C0020074A08B5536903F020
:104230000203536123B1054A93680BB1D0689847D4
:10424000BDE80840FFF746B9003C0140C84C0020DB
:10425000074A08B5536903F00403536123B1054AC3
:1042600013690BB150699847BDE80840FFF732B9B0
:10427000003C0140C84C0020074A08B5536903F0D0
:104280000803536123B1054A93690BB1D06998477C
:10429000BDE80840FFF71EB9003C0140C84C0020B3
:1042A000074A08B5536903F01003536123B1054A67
:1042B000136A0BB1506A9847BDE80840FFF70AB986
:1042C000003C0140C84C0020164B10B55C6904F45A
:1042D00078725A61A30604D5134A936A0BB1D06A67
:1042E0009847600604D5104A136B0BB1506B984782
:1042F000210604D50C4A936B0BB1D06B9847E205AD
:1043000004D5094A136C0BB1506C9847A30504D52A
:10431000054A936C0BB1D06C9847BDE81040FFF78D
:10432000D9B800BF003C0140C84C0020194B10B563
:104330005C6904F47C425A61620504D5164A136D27
:104340000BB1506D9847230504D5134A936D0BB1FB
:10435000D06D9847E00404D50F4A136E0BB1506E30
:104360009847A10404D50C4A936E0BB1D06E9847C0
:10437000620404D5084A136F0BB1506F98472304A9
:1043800004D5054A936F0BB1D06F9847BDE8104034
:10439000FFF7A0B8003C0140C84C002008B5FFF76B
:1043A0005DFEBDE80840FFF795B80000062108B59E
:1043B0000846FFF7B9F806210720FFF7B5F80621F0
:1043C0000820FFF7B1F806210920FFF7ADF8062114
:1043D0000A20FFF7A9F806211720FFF7A5F8062104
:1043E0002820FFF7A1F8BDE8084007211C20FFF7AF
:1043F0009BB8000008B5FFF745FE00F007F8FFF78F
:1044000007FEBDE80840FFF733BD00000023054A62
:1044100019460133102BC2E9001102F10802F8D14C
:10442000704700BFC84C00200B460146184600F0FC
:104430002DB8000000F040B8012838BF012010B5A9
:104440000446204600F030F830B900F007F808B90B
:1044500000F00CF88047F4E710BD0000024B18682C
:10446000BFF35B8F704700BF484D002008B50620A2
:1044700000F084F80120FFF7A3FA0000024B0A467F
:1044800001461868FFF7E2BB1C23002010B5054C5D
:1044900013462CB10A4601460220AFF3008010BD3E
:1044A0002046FCE700000000024B01461868FFF7B9
:1044B000D1BB00BF1C230020024B01461868FFF748
:1044C000CDBB00BF1C23002010B50139024490422F
:1044D00001D1002005E0037811F8014FA34201D07B
:1044E000181B10BD0130F2E72DE9F041A3B1C91A44
:1044F00017780144044603F1FF3C8C42204601D961
:10450000002009E00578BD4204F10104F5D10CEB6F
:104510000405D618A54201D1BDE8F08115F8018D3A
:1045200016F801EDF045F5D0E7E700001F2938B592
:1045300004460D4604D9162303604FF0FF3038BD02
:10454000426C12B152F821304BB9204600F030F8DD
:104550002A4601462046BDE8384000F017B8012B36
:104560000AD0591C03D1162303600120E7E7002479
:1045700042F82540284698470020E0E7024B0146D4
:104580001868FFF7D3BF00BF1C23002038B5074DC4
:1045900000230446084611462B60FFF715FA431C1A
:1045A00002D12B6803B1236038BD00BF4C4D002001
:1045B000FFF704BA034611F8012B03F8012B002A78
:1045C000F9D1704773772D626F6F6D2D6634303778
:1045D0002D626C0040A2E4F1646891060041A3E5FD
:1045E000F2656992070000004261642043414E4930
:1045F0006661636520696E6465782E008000000046
:1046000000800000000080000000000000000000AA
:1046100095190008B521000811210008D5190008D6
:10462000E1190008E11B0008A5190008B5190008E8
:10463000A9190008B1190008AD190008051B0008E8
:10464000B919000885240008C9190008D91A0008FA
:104650006330000050460008804A0020904C002043
:10466000004000000040000000400000004000004A
:104670000000010000000200000002000000020033
:104680006D61696E0069646C6500000000040028BB
:1046900000000000AAAAAAAA00000024FFFF000050
:1046A00000000000000000000000100000000000FA
:1046B000AAAA9AAA00000000FFFB00000000000068
:1046C000000000000000011000000000AAAAAA9A41
:1046D00000000000FFFE00000000000000000000DD
:1046E0000A04004000000000AAA6AAAA00000000D8
:1046F000DF7F0000990000000000000000000000C3
:1047000000000000AAAAAAAA00000000FFFF000003
:104710000000000000000000000000000000000099
:10472000AAAAAAAA00000000FFFF000000000000E3
:10473000000000000000000000000000AAAAAAAAD1
:1047400000000000FFFF000000000000000000006B
:1047500000000000000000000A000000000000004F
:104760000300000000000000000000000000000046
:104770000000000000000000000000000000000039
:1047800000000000000000007117000000000000A1
:10479000000007000000000040420F00FE2A010058
:1047A000D2040000202300200000000000000000D0
:1047B00000000000000000000000000000000000F9
:1047C00000000000000000000000000000000000E9
:1047D00000000000000000000000000000000000D9
:1047E00000000000000000000000000000000000C9
:1047F00000000000000000000000000000000000B9
:084800000000000000000000B0
:00000001FF
